:020000040000FA
:2B000000FFFF62FF2500FFFFFFFFFFFFFFFFFFFFFFFFFFFFFFFFFFFFFFFFFFFFFFFFFFFFFFFFFFFFFFFFFFFFFFFFFF76
:2B002B00C01D966119DCC11DDCC175077758067718DC0100000000705D7719DCC11D167770876118DC6118DC6100AF54
:2B005600A0100EE1100AA1100AA1288442388442100A0100000000288AE2100AA1108E42280441100A41100A4180E8A9
:2B008100000000000000000000000000000000000000000000000000000000000000000000000000000000000080E7ED
:2B00AC00000000000000000000000000000000000000000000000000000000000000000000000000000000000080E7C2
:2B00D700000008800000000000000000002001000000000000000000008000000000090000000000000000000080F458
:2B010200000002810000000000000000000000000000000000000000003000000000020000000000000000000000CF4E
:2B012D00000000000000000000000000000000000000000000000000000000000000000000000000000000000080E740
:2B015800100000000000000000000000000000000000000000000000000000000000000000000000000000000080F7F5
:2B018300000000000000000000000000000000000000000000000000000000000000000000000000000000000080E7EA
:2B01AE00000000000000000000000000000000000000000000000000000000000000000000000000000000000080E7BF
:2B01D900000000000000000000000000000000000040000000000000000000000000000000000000000000000008AB08
:2B020400000000000000000000000000000000000000000000000000000000000000000000000000000000000080E768
:2B022F00000000000000000000000000000000000000000000000000000000000000000000000000000000000080E73D
:2B025A00000000000000000000000000000000000000000000000000000000000000000000000000000000000080E712
:2B028500000000000000000000000000000000000000000000000000000000000000000000000000000000000080E7E7
:2B02B000100000000000000000000000000000000010000000000000000400000000000000000000000000000008AA4D
:2B02DB00000000000000000000000000000000000000000000000000000000000000000000000000000000000080E791
:2B030600000000000000000000000000000000000000000000000000000000000000000000000000000000000080E765
:2B033100000000000000000000000000000000000020000000000000000400010000000000000000000000000080807C
:2B035C00000000000000000000000000000000000040000000000000000840000000000000000000000000000000E707
:2B0387002000000000000000004000000000000000000800000000080200080000000000000000000000000000808DC4
:2B03B20022000000000000000040000000000000000002000000000800000000000000000000000000000000008887A5
:2B03DD00020000000000000000000000000000000000000000000000000001000000000000000000000000000080F57D
:2B040800040000000000000000000000000000000000000000000000020000000000000000000000000000000080E162
:2B043300020000000000000000000000000000000000080000000000000008000000000000000000000000000000E5A7
:2B045E00020000000000000000000000000000000000000000000000000000000000000000000000000000000080E50C
:2B048900020000000000000000000000000000000000000000000000000000000000000000000000000000000008ED51
:2B04B400800008800008800008800008800008800008000000000020000220000220000220000220000220000280E7BA
:2B04DF00800008800008800008800008800008800008000000000020000220000220000220000220000220000280E78F
:2B050A00000000000000000000000000000000000000000000000000000000000000000000000000000000000080E75F
:2B05350000000000000000000000000000000000007E000000000000802100000000000000000000000000000080E319
:2B056000020000000000000000000000000000000018020000000000004000000000000000000000000000000088F29A
:2B058B00020000000000000000000000000000000024000000000000000700000000000000000000000000000008F818
:2B05B600020000000000000000000000000000000018000000000000000000000000000000000000000000000088F484
:2B05E1000200000000000000000000000000000000000200000000000046000000000000000000000000000000088D10
:2B060C0000000000000000000000000000000000000000000000000000060000000000000000000000000000008081BC
:2B06370000000000000000000000000000000000001800000000000000060000000000000000000000000000000098E2
:2B066200000000000000000000000000000000000000000000000000000000020000000000000000000000000080E506
:2B068D0000000000000000000000000000000000009E0000000000000000180000000000000000000000000000008705
:2B06B800000000000000000000000000000000000018080000000000000080000000000000000000000000000008FE71
:2B06E3000200000000000000000000000000000000040000000000000000F0000000000000000000000000000000D224
:2B070E00020000000000000000000000000000000018000000000000000000200000000000000000000000000000DCAA
:2B0739000200000000000000000000000000000000200200000000000000E0000000000000000000000000000000A3EE
:2B0764000200000000000000000000000000000000000000000000000000600000000000000000000000000000808305
:2B078F0000000000000000000000000000000000001800000000000000006000000000000000000000000000008890AF
:2B07BA00000000000000000000000000000000000000000000000000000000010000000000000000000000000080E6AD
:2B07E500000000000000000000000000000000000000000000000000000018000000000000000000000000000000FED3
:2B081000000000000000000000000000000000000000000000000000000000000000000000000000000000000080E756
:2B083B000000000000000000000000000000000000000000000000000000700800000000000000000000000000089082
:2B086600020000000000000000000000000000000000000000000000000000040000000000000000000000000008E970
:2B0891000200000000000000000000000000000000000000000000000000E000000000000000000000000000001092B8
:2B08BC000200000000000000000000000000000000000000000000000000600000000000000000000000000000088B1C
:2B08E7000200000000000000000000000000000000000000000000000000600000000000000000000000000000088BF1
:2B091200000000000000000000000000000000000040000000000000001000010000000000000000000000000008ABB6
:2B093D00000000000000000000000000000000000006000000000000800178000000000000000000000000000080E12F
:2B096800000000000000000000000000000000000000000000000000000860000000000000000000000000000000817B
:2B09930000000000000000000000000000000000003C010000000000000F10080000000000000000000000000080F362
:2B09BE00000000000000000000000000000000000000010000000000000064040000000000000000000000000008CCD1
:2B09E900020000000000000000000000000000000018000000000000000E800000000000000000000000000000889221
:2B0A14000200000000000000000000000000000000180000000000000006000000000000000000000000000000108BFC
:2B0A3F00020000000000000000000000000000000018000000000000000660000000000000000000000000000088F490
:2B0A6A00020000000000000000000000000000000000100000000000000000000000000000000000000000000008FD4A
:2B0A950000000000000000000000000000000000002600000000000080011C400000000000000000000000000008AD7E
:2B0AC000000000000000000000000000000000000020000000000000008000040000000000000000000000000080C91E
:2B0AEB0000000000000000000000000000000000003C0000000000000007700000000000000000000000000000009C91
:2B0B1600000000000000000000000000000000000000020000000000000800000000000000000000000000000000E5C5
:2B0B41000200000000000000000000000000000000180000000000000006E0080000000000000000000000000008FC7D
:2B0B6C00020000000000000000000000000000000018000000000000000660000000000000000000000000000088F462
:2B0B9700040000000000000000000000000000000018000000000000000660000000000000000000000000000010EBB6
:2B0BC200020000000000000000000000000000000000100000000000001000000000000000000000000000000008FCE2
:2B0BED0002000000000000000000000000000000003E0000000000008007F8020000000000000000000000000008B460
:2B0C1800020000000000000000000000000000000038000000000000000EE0000000000000000000000000000088D62B
:2B0C430000000000000000000000000000000000002400000000000000091000000000000000000000000000000085C4
:2B0C6E00000000000000000000000000000000000018020000000000000664400000000000000000000000000000FC9B
:2B0C9900000000000000000000000000000000000000000000000000000880000000000000000000000000000080E741
:2B0CC400020000000000000000000000000000000000000000000000000000000000000000000000000000000008ED0E
:2B0CEF00020000000000000000000000000000000018000000000000000660000000000000000000000000000088F4DE
:2B0D1A00040000000000000000000000000000000040000000000000008000000000000000000000000000000090BE9C
:2B0D4500020000000000E0830000000000000000001E000000000000800798020000000000000000000000000088A3B4
:2B0D7000020000000000800300000000000000000018000000000000000680000000000000000000000000000088A904
:2B0D9B00020000000000400000000000000000000024010000000000000174000000000000000000000000000008E861
:2B0DC600000000000000800100000000000000000018010000000000000E00400000000000000000000000000000C05A
:2B0DF1000000000000000042000000000000000000000000000000000000E0000000000000000000000000000000A70E
:2B0E1C00000000000000000000000000000000000000000000000000000060000000000000000000000000000080814A
:2B0E4700020000000000800100000000000000000018000000000000000660000000000000000000000000000008ED8A
:2B0E7200020000000000000000000000000000000000000000000000000000020000000000000000000000000008EF5A
:2B0E9D00040000000000608200000000000000000086000000000000802778000000000000000000000000000010DAB5
:2B0EC8000200000000000002000000000000000000000800000000000046E0000000000000000000000000000088C382
:2B0EF300020000000000C0010000000000000000001C000000000000000190000000000000000000000000000088EDEF
:2B0F1E00020000000000000000000000000000000000000000000000000660200000000000000000000000000008CD4B
:2B0F4900000000000000804300000000000000000038020000000000004080000000000000000000000000000000E5DB
:2B0F7400000000000000800100000000000000000018000000000000000000000000000000000000000000000080E752
:2B0F9F000E00000000008001000000000000000000180000000000000006600000000000000000000000000000A0CBAF
:2B0FCA00100000000000000000000000000000000000000000000000000000000000000000000000000000000080F775
:2B0FF500000000000000000000000000000000000000000000000000000000000000000000000000000000000080E76A
:2B102000800008800008800008800008800008800008000000000020000220000220000220000220000220000280E742
:2B104B00800008800008800008800008800008800008000000000020000220000220000220000220000220000280E717
:2B1076000000000000000004500000000000000000A4000000000000002108000003000000000000000000000080BFEC
:2B10A100000000000000000000000000000000000000000000000000000000000000000000000000000000000080E7BD
:2B10CC00000000000000200002000000000000080000000000000000000440000000000000000010000000000080FEFD
:2B10F700000800000000000000001000000000000000000000000000000000022000002000000000000000000000E490
:2B1122000008000000002004420010000000000800A4000000000000002108022002002000000010000000000000A457
:2B114D00000000000000000000000000000000000008000000000000000184000000000000000000000000000080BEAC
:2B11780000000000000000000000000000000000002400000000000000002200000000000000000000000000008087FF
:2B11A300000000000000000800000000000000000000000000000000000000400000000000000000000000000000A732
:2B11CE00000000000000000000000000000000000000000000000000000010100000000000000000000000000080E670
:2B11F9000C00000000004000000000000000000000000000000000000000000000000000000000000000000000E0CDD2
:2B122400000000000000000000000000000000000000000000000000000100000000000000000000000000000080F628
:2B124F00020000000000000000000000000000000000000000000000000000000000000000000000000000000080E50D
:2B127A00000000000000000000000000000000000000080000000000000000000000000000000000000000000080EFD2
:2B12A500000000000000000000000000000000000000000000000000000000000000000000000000000000000080E7B7
:2B12D0000C0000000000000000000000000000000000000000000000000000000000000000000000000000000080EB7C
:2B12FB00000000000000004000000000000000000000000000000000000010000000000000000000000000000080F206
:2B132600000000000000000000000000000000000000000000000000000000200000000000000000000000000008CFA5
:2B1351000000000000000000000000000000000000000000000000000000000000000000000000000000000000E08110
:2B137C00000000000000000000000000000000000000020000000000000000000000000000000000000000000090F4C0
:2B13A700000000000000000000000000000000000000000000000000000000000000000000000000000000000080E7B4
:2B13D200000000000000000000000000000000000000000000000000000000000000000000000000000000000080E789
:2B13FD00000000000000000000000000000000000000000000000000000000000000010000000000000000000080E65E
:2B142800000000000000000000000000000000000000000000000000000000000040001000000000000000000080A227
:2B1453000000000000000000000000000000000000000000000000000000000000000000000000000000000000F090EE
:2B147E00000000000000000000000000000000000000000000000000000000000000000000000000000000000080E7DC
:2B14A900000000000000000000000000000000000000000000000000000000000000000000000000000000000080E7B1
:2B14D400000000000000000000000000000000000000000000000000000000000000000000000000000000000080E786
:2B14FF00000000000000000000000000000000000000000000000000000000000000000000000000000000000008EFCB
:2B152A00000000000000000000000000000000000000000000000000000000000000018000000000000000000078910C
:2B155500000000000000000000000000000000000000000000000000000000000000000000000000000000000080E704
:2B158000000000000000000000000000000000000000000000000000000000000000000000000000000000000080E7D9
:2B15AB00000000000000000000000000000000000000000000000000000000000000000000000000000000000080E7AE
:2B15D600000000000000000000000000000000000000000000000000000000000000000000000000000000000080E783
:2B160100000000000000000000000000000000000000000000000000800000002040A02900000000020000020000927F
:2B162C00020000000000000000000000000000000000000000000000800000000000800000000000000000000008ED9C
:2B165700000000000000000000000000000000000000000000000000000000000000000001000000000000000008FF60
:2B168200000000000000000000000000000000000000000000000000000000002040000000000000020000020090B099
:2B16AD00000000000000000000000000000000000000000000000000000000000000202900000000000000000088DC65
:2B16D800000000000000000000000000000000000000000000000000000000000000000000000000000000000008EFF0
:2B170300020000000000000000000000000000000000000000000000000000000000000000000000000000000008EDC4
:2B172E00800008800008800008800008800008800008000000000020000220000220000220000220000220000280E72D
:2B175900800008800008800008800008800008800008000000000020000220000220000220000220000220000280E702
:2B178400000000000000000000000000000000000000000000000000000000000000001000000000000000000080E6C4
:2B17AF000000000000000000000000000000000000000000000000000000000000F88201000000000000000000888B81
:2B17DA00020000000000000000000000000000000000000000000000000000000060048000000000000000000008876F
:2B180500020000000000000000000000000000000000000000000000000000000010000F0000000000000000001092F5
:2B183000020000000000000000000000000000000000000000000000000000000060400000000000000000000008CB18
:2B185B00020000000000000000000000000000000000000000000000000000000080004E000000000000000000088FFB
:2B18860000000000000000000000000000000000000000000000000000000000000000060000000000000000000889A0
:2B18B100000000000000000000000000000000000000000000000000000000000060000600000000000000000080E73F
:2B18DC00000000000000000000000000000000000000000000000000000000000000001000000000000000000080E66B
:2B1907000000000000000000000000000000000000000000000000000000000000188207000000000000000000808311
:2B193200000000000000000000000000000000000000000000000000000000000000008600000000000000000008817B
:2B195D000200000000000000000000000000000000000000000000000000000000F00409000000000000000000088FC9
:2B1988000200000000000000000000000000000000000000000000000000000000000806000000000000000000909AFA
:2B19B3000200000000000000000000000000000000000000000000000000000000600048000000000000000000888F48
:2B19DE000200000000000000000000000000000000000000000000000000000000600000000000000000000000088BE9
:2B1A0900000000000000000000000000000000000000000000000000000000000060000600000000000000000008EF55
:2B1A3400000000000000000000000000000000000000000000000000000000000000001000000000000000000080E611
:2B1A5F00000000000000000000000000000000000000000000000000000000000078820F00000000000000000000E56E
:2B1A8A00000000000000000000000000000000000000000000000000000000000060000600000000000000000080E764
:2B1AB500000000000000000000000000000000000000000000000000000000000090040904000000000000000008ABB2
:2B1AE000020000000000000000000000000000000000000000000000000000000060080601000000000000000008F56D
:2B1B0B00020000000000000000000000000000000000000000000000000000000000000800000000000000000010F4A1
:2B1B3600020000000000000000000000000000000000000000000000000000000000000000000000000000000008ED8D
:2B1B6100020000000000000000000000000000000000000000000000000000000060000600000000000000000008EDFC
:2B1B8C00000000000000000000000000000000000000000000000000000000000000010000000000000000000008EE37
:2B1BB700000000000000000000000000000000000000000000000000000000000018804700000000000000000080851F
:2B1BE200000000000000000000000000000000000000000000000000000000000080000E000000000000000000808149
:2B1C0D00000000000000000000000000000000000000000000000000000000000070000100000000000000000080813A
:2B1C38000000000000000000000000000000000000000000000000000000000000000046000000000000000000088DA6
:2B1C63000200000000000000000000000000000000000000000000000000000000E008080000000000000000000883D9
:2B1C8E0002000000000000000000000000000000000000000000000000000000006000000000000000000000009092A7
:2B1CB900020000000000000000000000000000000000000000000000000000000060000600000000000000000008EDA3
:2B1CE400020000000000000000000000000000000000000000000000000000000000040000000000000000000008E9DE
:2B1D0F00000000000000000000000000000000000000000000000000000000000098801100000000000000000088EE0A
:2B1D3A00000000000000000000000000000000000000000000000000000000000000000800000000000000000000E78F
:2B1D6500000000000000000000000000000000000000000000000000000000000070040F00000000000000000000E3ED
:2B1D9000000000000000000000000000000000000000000000000000000000000000080002000000000000000080CFCF
:2B1DBB000000000000000000000000000000000000000000000000000000000000E0000600000000000000000088EFA0
:2B1DE600020000000000000000000000000000000000000000000000000000000060000600000000000000000080E505
:2B1E1100020000000000000000000000000000000000000000000000000000000060000600000000000000000080E5D9
:2B1E3C00020000000000000000000000000000000000000000000000000000000000011000000000000000000080E503
:2B1E670002000000000000000000000000000000000000000000000000000000007880090000000000000000000083CA
:2B1E92000000000000000000000000000000000000000000000000000000000000E00000000000000000000000888934
:2B1EBD00000000000000000000000000000000000000000000000000000000000010000F04000000000000000000C116
:2B1EE800000000000000000000000000000000000000000000000000000000000060000001000000000000000080915D
:2B1F1300000000000000000000000000000000000000000000000000000000000080080E000000000000000000808904
:2B1F3E0000000000000000000000000000000000000000000000000000000000000000060000000000000000000889E1
:2B1F6900020000000000000000000000000000000000000000000000000000000060000600000000000000000008EDF0
:2B1F9400020000000000000000000000000000000000000000000000000000000000000000000000000000000090F49C
:2B1FBF00020000000000000000000000000000000000000000000000000000000098824100000000000000000088EB27
:2B1FEA00020000000000000000000000000000000000000000000000000000000000040800000000000000000088E94D
:2B201500000000000000000000000000000000000000000000000000000000000070000700000000000000000008EF32
:2B204000000000000000000000000000000000000000000000000000000000000000404000000000000000000080A3D2
:2B206B000000000000000000000000000000000000000000000000000000000000E0000E00000000000000000080E7F5
:2B209600000000000000000000000000000000000000000000000000000000000060000600000000000000000080E752
:2B20C100000000000000000000000000000000000000000000000000000000000060000600000000000000000008EF97
:2B20EC00020000000000000000000000000000000000000000000000000000000000040000000000000000000008E9D2
:2B2117000200000000000000000000000000000000000000000000000000000000F8801700000000000000000010F507
:2B214200020000000000000000000000000000000000000000000000000000000060000E00000000000000000088ED8D
:2B216D00020000000000000000000000000000000000000000000000000000000010040900000000000000000088E9B7
:2B219800000000000000000000000000000000000000000000000000000000000060080602000000000000000008C7DD
:2B21C300000000000000000000000000000000000000000000000000000000000080000000000000000000000000E78A
:2B21EE00000000000000000000000000000000000000000000000000000000000000000000000000000000000080E75F
:2B2219000E0000000000000000000000000000000000000000000000000000000060000600000000000000000080E9BD
:2B2244001E0000000000000000000000000000000000000000000000000000000000000000000000000000000080F9D8
:2B226F00000000000000000000000000000000000000000000000000000000000000000000000000000000000080E7DD
:2B229A00800008800008800008800008800008800008000000000020000220000220000220000220000220000280E7B6
:2B22C500800008800008800008800008800008800008000000000020000220000220000220000220000220000280E78B
:2B22F000000000000000000000000000000000000000000000000000000000000080800C030000000000000000009B19
:2B231B00000000000000000000000000000000000000000000000000000000000000000000000000000000000080E730
:2B234600000000000000000000000000000000000000000000000000000000000000000000000000000000000080E705
:2B237100000000000000000000000000000000000000000000000000000080000000000000020000002000022000E796
:2B239C00000000000000000000000000000000000000000000000000000080000080800802020000002000022080CFF9
:2B23C700000000000000000000000000000000000000000000000000000000000040000000000000000000000080A388
:2B23F200000000000000000000000000000000000000000000000000000000000080000200000000000000000000C579
:2B241D00000000000000000000000000000000000000000000000000000000000020000100000000000000000080D41F
:2B244800000000000000000000000000000000000000000000000000000000000000000100000000000000000080F6F2
:2B247300000000000000000000000000000000000000000000000000000000000010000400000000000000000058EFE3
:2B249E00000000000000000000000000000000000000000000000000000000000020000000000000000000000080C5AE
:2B24C900000000000000000000000000000000000000000000000000000000000000000000000000000000000008EFF1
:2B24F400000000000000000000000000000000000000000000000000000000000000000000000000000000000080E756
:2B251F00000000000000000000000000000000000000000000000000000000000000000000000000000000000080E72A
:2B254A000000000000000000000000000000000000000000000000000000000000000000000000000000000000D0B2E4
:2B257500000000000000000000000000000000000000000000000000000000000000000202000000000000000080E5D2
:2B25A000000000000000000000000000000000000000000000000000000000000000200000000000000000000080C7A9
:2B25CB00000000000000000000000000000000000000000000000000000000000000000000000000000000000080E77E
:2B25F600000000000000000000000000000000000000000000000000000000000000002000000000000000000080E535
:2B2621001C0000000000000000000000000000000000000000000000000000000000000000000000000000000008F377
:2B264C00000000000800000000000000000000000000000000000000000000000000000000000000000000000000E774
:2B2677000000000000000000000000000006000000000000000000000000000000000000000001000000000000809021
:2B26A200000000000000000000000000000000000000000000000000000000000000000000000000000000000080E7A6
:2B26CD00000000000000000000000000000000000000000000000000000000000000000000000000000000000080E77B
:2B26F800000000000000000000000000000100000000000000000000000000000000000000000000000000000080F640
:2B272300000000000000000000000000000000000000000000000000000000000000000000000000000000000080E724
:2B274E000000000000000000000000000000000000000000000000000000000000000000000000000000000000C0A3FD
:2B277900002001000000000000000000000000000000000000000000000000000000000000000000000000000080F59F
:2B27A4000000000000000000000000000000000000000000000000000000000000000000000050000000000000C0A654
:2B27CF00000000000000000000000000000000000000000000000000000000000000000000000000000000000080E778
:2B27FA00000000000000000000000000000000000000000000000000000000000000000000000000000000000080E74D
:2B282500800100000000000000000000000000000000000000000000000000000000000000000000000000000000FE09
:2B285000000000000000000000000000000000000000000000000000000000000000000000000000000000000080E7F6
:2B287B000080000200022000040008800000A001000200000000000000000402000000000A800002000000000000ECE1
:2B28A600020000000002200004000000000000000002000000000000000004000000000008000000000000000088C584
:2B28D100020000000000000000000000004000000000000000000000000000000000000000000400000000000008ADE1
:2B28FC00040000000000000000000880000000010000000000000000000000020000000002000000000000000090D1BF
:2B2927000280000200000000000000000000B0020000000000000000000000000000000000800002000000000008FEC7
:2B295200020000000000000000000000000000000000000000000000000000000000000000000000000000000008ED63
:2B297D00020000000000000000000000000000000000000000000000000000000000000000000000000000000008ED38
:2B29A800800008800008800008800008800008800008000000000020000220000220000220000220000220000280E7A1
:2B29D300800008800008800008800008800008800008000000000020000220000220000220000220000220000280E776
:2B29FE00000000000000000000000000000400000000000000000000000000000000000000000000000000000080A387
:2B2A2900E20900000000000000000000E00300000000000000000000000000000000000000801700000000000080B9E4
:2B2A54008201000000000000000000008081000000000000000000000000000000000000000006000000000000088342
:2B2A7F004480000000000000000000004002000000000000000000000000000000000000000009040000000000889001
:2B2AAA0082810000000000000000000080210000000000000000000000000000000000000000060100000000000891BD
:2B2AD500020200000000000000000000000200000000000000000000000000000000000000000000000000000008EDDB
:2B2B0000020000000000000000000000000000000000000000000000000000000000000000000000000000000080E543
:2B2B2B008001000000000000000000008001000000000000000000000000000000000000000006000000000000808176
:2B2B5600000000000000000000000000000400000000000000000000000000000000000000001000000000000080A21E
:2B2B8100600800000000000000000000600200000000000000000000000000000000000000800100000000000080DC82
:2B2BAC00020000000000000000000000008000000000000000000000000000000000000000008000000000000080E597
:2B2BD700C28100000000000000000000C00300000000000000000000000000000000000000000F00000000000088B086
:2B2C0200048000000000000000000000002000000000000000000000000000000000000000000000000000000008E11A
:2B2C2D00820300000000000000000000800300000000000000000000000000000000000000000E02000000000088AB31
:2B2C58008201000000000000000000008001000000000000000000000000000000000000000006000000000000088BB4
:2B2C83008201000000000000000000008001000000000000000000000000000000000000000006000000000000808319
:2B2CAE00000000000000000000000000000000000000000000000000000000000000000000001000000000000080E685
:2B2CD900E00B00000000000000000000E00700000000000000000000000000000000000000800700000000000080DC1B
:2B2D04008001000000000000000000008001000000000000000000000000000000000000000086000000000000808913
:2B2D2F00402000000000000000000000400201000000000000000000000000000000000000000900000000000088CE77
:2B2D5A00820300000000000000000000800100000000000000000000000000000000000000000600000000000008A991
:2B2D8500020200000000000000000000000001000000000000000000000000000000000000000802000000000010E61E
:2B2DB000020000000000000000000000000000000000000000000000000000000000000000000000000000000008ED01
:2B2DDB008201000000000000000000008001000000000000000000000000000000000000000006000000000000088B30
:2B2E0600000400000000000000000000001000000000000000000000000000000000000000000800000000000088AA53
:2B2E3100600000000000000000000000E0010000000000000000000000000000000000000080070000000000008081AD
:2B2E5C000000000000000000000000008001000000000000000000000000000000000000000046000000000000009CE8
:2B2E8700C01300000000000000000000402000000000000000000000000000000000000000000900000000000080CE96
:2B2EB2000200000000000000000000008041000000000000000000000000000000000000000046000000000000009A52
:2B2EDD00820101000000000000000000000200000000000000000000000000000000000000000000000000000088C6F6
:2B2F0800840100000000000000000000000000000000000000000000000000000000000000000000000000000088F29F
:2B2F33008201000000000000000000008001000000000000000000000000000000000000000006000000000000088BD6
:2B2F5E00021000000000000000000000000000000000000000000000000000000000000000000000000000000008EC42
:2B2F8900620200000000000000000000E00B00000000000000000000000000000000000000801100000000000000E459
:2B2FB400000000000000000000000000800100000000000000000000000000000000000000000000000000000000FE73
:2B2FDF00C01100000000000000000000402200000000000000000000000000000000000000000F04000000000080E819
:2B300A00008000000000000000000000800300000000000000000000000000000000000000000001000000000000C4D3
:2B303500800100000000000000000000000200000000000000000000000000000000000000000600000000000000BA2D
:2B30600082010000000000000000000000000000000000000000000000000000000000000000060000000000008892A2
:2B308B008201000000000000000000008001000000000000000000000000000000000000000006000000000000088B7D
:2B30B600020400000000000000000000000000000000000000000000000000000000000000000800000000000088A9B0
:2B30E100E20100000000000000000000600A00000000000000000000000000000000000000800100000000000088CF9F
:2B310C00800100000000000000000000000000000000000000000000000000000000000000004000000000000000FADD
:2B313700401200000000000000000000C02300000000000000000000000000000000000000000F000000000000808A1F
:2B316200800100000000000000000000000200000000000000000000000000000000000000004000000000000000D8A7
:2B318D00000001000000000000000000800300000000000000000000000000000000000000000600000000000000AAE3
:2B31B8000200000000000000000000008001000000000000000000000000000000000000000006000000000000009AC9
:2B31E3008201000000000000000000008001000000000000000000000000000000000000000006000000000000088B24
:2B320E00040000000000000000000000000000000000000000000000000000000000000000000000000000000008EB9E
:2B323900620A00000000000000000000600600000000000000000000000000000000000000802900000000000088B2B5
:2B326400020000000000000000000000000000000000000000000000000000000000000000000000000000000008ED48
:2B328F00C22100000000000000000000C00301000000000000000000000000000000000000004700000000000080A600
:2B32BA00000200000000000000000000000000000000000000000000000000000000000000000000000000000080C5A2
:2B32E500800300000000000000000000800101000000000000000000000000000000000000004E00000000000000B7B4
:2B3310008001000000000000000000008001000000000000000000000000000000000000000006000000000000808189
:2B333B0080010000000000000000000080010000000000000000000000000000000000000000060000000000000889CE
:2B336600021000000000000000000000001000000000000000000000000000000000000000000000000000000008ED25
:2B339100E20300E00101000000000000600000000000000000000000000000000000000000802F00000000000090DBD0
:2B33BC008201008041000000000000000000000000000000000000000000000000000000000006000000000000088F05
:2B33E700421000400200000000000000C0210000000000000000000000000000000000000000410000000000008880FD
:2B3412008081008001010000000000000040000000000000000000000000000000000000000006000000000000089529
:2B343D00000000000200000000000000800300000000000000000000000000000000000000004800000000000080FA1D
:2B346800000000000000000000000000800100000000000000000000000000000000000000000000000000000000FEBA
:2B349300820100800100000000000000800100000000000000000000000000000000000000000600000000000030A9AA
:2B34BE000A00000000000000000000000000000000000000000000000000000000000000000000000000000000F09A4F
:2B34E900000000000000000000000000000000000000000000000000000000000000000000000000000000000080E751
:2B351400800008800008800008800008800008800008000000000020000220000220000220000220000220000280E729
:2B353F00800008800008800008800008800008800008000000000020000220000220000220000220000220000280E7FE
:2B356A00000230000000000000000000008000040000000000000000000000000000000000801000000000000000F3FD
:2B359500000000000000000000000000000000000000000000000000000000000000000000000000000000000080E7A4
:2B35C000000002400000000000000000200002240000000000000000000000000000000000000000000000800000AB2D
:2B35EB00002000800000000080000080000000000000000000000000000000000000020000000000000000000000EF24
:2B361600000222400000000080000080208002200000000000000000000000000000020000801000000000800080AC25
:2B364100000200000000000000000000000000000000000000000000000000000000000000000600000000000080A333
:2B366C0000000000000000000000000040000000000000000000000000000000000000000000020000000000008085EC
:2B369700000000000000000000000000000000000000000000000000000000000000000000000003000000000080D7AE
:2B36C200000000000000000000000000004400000000000000000000000000000000000000000000000000000080A772
:2B36ED00000000000001000000000000008000000000000000000000000000000000000000000000000000000008F732
:2B371800106000000000000000000000000000000000000000000000000000000000000000000000000000000080F1A5
:2B374300000000000000000000000000000000000000000000000000000000000000000000000000000000000080E7F4
:2B376E00800000000000000000000000000000000000000000000000000000000000000000000000000000000000EFC1
:2B379900000000000000000000000000000001000000000000000000000000000000000000000000000000000080F78D
:2B37C400000000000000000000000000000000000000000000000000000000000000000000000000000000000080E773
:2B37EF00000000000000000000000000000000000000000000000000000000000000000000000000000000000080E748
:2B381A00440000008000000000000000000000000000000000000000000000000000000000000400000000000080EF4C
:2B384500000000000000000000000000000000000000000000000000000000000000000000000000000000000008EF61
:2B387000000000000000000000000000000800000000000000000000000000000000000000000000000000000000E73E
:2B389B00004000000000000000000000000000000080010000000000000000000000000000002800000000000080E0B9
:2B38C600800000000000000000000000000000000000020000000000000000000000000000008000000000000000E5F0
:2B38F100000000000000000000000000000000000000000000000000000000000000000000000000000000000080E745
:2B391C00000000000000000000000000000000000000000000000000000000000000000000000000000000000080E719
:2B394700E0280AA11004A1108A422884A2100AA110840300000000100441100AA1100AA1100AE12804A1108AA200AFF3
:2B3972006071DDC11D86C11D5C777007D71DDCC11D86050000000018866118DCC11DDCC11DDC617187C11D5CD7059F42
:02399D00FFFF2A
:00000001FF
